:020000040000FA
:1000000001288B01831603139B018117FC308600A6
:100010000730831203139000861420140E1C201046
:1000200020181528701C17281928701C192806106C
:100030001B2806140000031083120313A00DA10D4A
:10004000A20DA30DA40DA50DA60DA70DA80DA90D1C
:10005000AA0DAB0DAC0DAD0DAE0DAF0DB00DB10DCC
:10006000B20DB30DB40DB50DB60DB70DB80DB90D7C
:10007000BA0DBB0DBC0DBD0DBE0DBF0DC00DC10D2C
:10008000C20DC30DC40DC50DC60DC70DC80DC90DDC
:10009000CA0DCB0DCC0DCD0DCE0DCF0DD00DD10D8C
:1000A000D20DD30DD40DD50DD60DD70DD80DD90D3C
:1000B000DA0DDB0DDC0DDD0DDE0DDF0DE00DE10DEC
:1000C000E20DE30DE40DE50DE60DE70DE80DE90D9C
:1000D000EA0DEB0DEC0DED0DEE0DEF0D8316031398
:1000E000A00DA10DA20DA30DA40DA50DA60DA70D8C
:1000F000A80DA90DAA0DAB0DAC0DAD0DAE0DAF0D3C
:10010000B00DB10DB20DB30DB40DB50DB60DB70DEB
:10011000B80DB90DBA0DBB0DBC0DBD0DBE0DBF0D9B
:10012000C00DC10DC20DC30DC40DC50DC60DC70D4B
:10013000C80DC90DCA0DCB0DCC0DCD0DCE0DCF0DFB
:10014000D00DD10DD20DD30DD40DD50DD60DD70DAB
:10015000D80DD90DDA0DDB0DDC0DDD0DDE0DDF0D5B
:10016000E00DE10DE20DE30DE40DE50DE60DE70D0B
:10017000E80DE90DEA0DEB0DEC0DED0DEE0DEF0DBB
:1001800083120317900D910D920D930D940D950D03
:10019000960D970D980D990D9A0D9B0D9C0D9D0D2B
:1001A0009E0D9F0DA00DA10DA20DA30DA40DA50DDB
:1001B000A60DA70DA80DA90DAA0DAB0DAC0DAD0D8B
:1001C000AE0DAF0DB00DB10DB20DB30DB40DB50D3B
:1001D000B60DB70DB80DB90DBA0DBB0DBC0DBD0DEB
:1001E000BE0DBF0DC00DC10DC20DC30DC40DC50D9B
:1001F000C60DC70DC80DC90DCA0DCB0DCC0DCD0D4B
:10020000CE0DCF0DD00DD10DD20DD30DD40DD50DFA
:10021000D60DD70DD80DD90DDA0DDB0DDC0DDD0DAA
:10022000DE0DDF0DE00DE10DE20DE30DE40DE50D5A
:10023000E60DE70DE80DE90DF00D831203133830DC
:0E024000FF3E031D2029000086100C28090037
:02400E00623F0F
:02401000FC3F73
:00000001FF
